:100000000C9417060C9499280C94C6280C943F065F
:100010000C943F060C94B20C0C943F060C943F06D3
:100020000C943F060C943F060C943F060C943F063C
:100030000C943F060C943F060C943F060C943F062C
:100040000C94F3280C943F060C948B2C0C94C62C27
:100050000C943F060C943F060C943F060C943F060C
:100060000C943F060C943F06EE1BF51BF51BEE1B94
:10007000F51BF51BF51BF51BF51BF51BF51BF51B00
:10008000F51BF51BF51BF51BF51B631BF51BF51B82
:10009000F51BF51BF51BC61AF51BF51BF51BF51B10
:1000A000F51BF51BF51BF51BF51BF51BF51BF51BD0
:1000B000F51BF51BF51B6F1B6F1B6F1B6F1B6F1B5E
:1000C0006F1B6F1B6F1B6F1BF51BF51BF51BF51BC8
:1000D000F51BF51BCB1A6E1B6E1B6E1B6E1BF51BE7
:1000E0007F1B871B8F1B971B9F1BA71BAF1BB71B60
:1000F000C11BCB1BD51BDF1B121BD21AF51BF51B1B
:10010000F51BF51B631BF51BF51BF51BF51BF51B01
:10011000F51BF51BF51B6D1B6D1B6D1B6D1BF51B7F
:100120007F1B871B8F1B971B9F1BA71BAF1BB71B1F
:10013000C11BCB1BD51BDF1B121BD21AF51BF51BDA
:10014000F51BF51B631B261C261C261C261C261CC7
:10015000261C261C261C261C261C261C261C261C8F
:10016000471D471D471D471D471D471D6D1C771C1B
:10017000811C8B1CF11CFB1C091D1B1DB81D281E9E
:10018000F91DFE1D031E081E0D1E121E171E281E21
:10019000221E35254A2556255F256C2592259A2550
:1001A000BD25AA25456E746572206D656E752E2E6F
:1001B0002E00546F67676C6564206D6963726F50C1
:1001C000504D00546F67676C656420696E76657288
:1001D0007465642050504D2100546F67676C6564EE
:1001E000205458206D7574696E672100546F6767DD
:1001F0006C65642074656C656D657472792100505E
:10020000726F746F636F6C206572726F72207769A2
:1002100074682052580054696D656F757420776852
:10022000656E20636F6E6E656374696E6720746FB0
:1002300020525800507265737320616E79206B658F
:100240007920746F2063616E63656C00436F6E6E1E
:10025000656374696E6720746F2052582C20706F2C
:100260007765722075702074686520525820287751
:100270006974682062696E6420706C7567206966B5
:10028000206E6F74207573696E6720616C77617979
:10029000732062696E642900546F67676C6564201F
:1002A00027696D6D656469617465206F757470751B
:1002B000742700546F67676C65642027736C6176E0
:1002C00065206D6F64652700546F67676C656420F7
:1002D00027616C776179732062696E642700546FBF
:1002E00067676C65642050504D206368616E6E6571
:1002F0006C206C696D6974005365742052535349C6
:1003000020696E6A656374696F6E206368616E6EE2
:10031000656C2028303D3D64697361626C6529001D
:100320005365742050504D206D696E696D756D2058
:1003300073796E630053657420626561636F6E202C
:10034000696E74657276616C0053657420626561D4
:10035000636F6E2064656C6179005365742062651B
:1003600061636F6E206672657175656E6379206971
:100370006E20487A3A20303D64697361626C652C66
:100380002050783D504D52206368616E6E656C2040
:10039000782C2046783D465253206368616E6E6526
:1003A0006C2078005365742050574D2073746F7023
:1003B0002064656C61792028302064697361626C07
:1003C00065642C20312D323535203D3D20302E31D5
:1003D00073202D2035306D696E29005365742050CF
:1003E000504D2073746F702064656C6179202830E3
:1003F0002064697361626C65642C20312D3235355F
:10040000203D3D20302E3173202D2035306D696E1A
:100410002900536574206661696C736166652064A8
:10042000656C61792028302064697361626C656451
:100430002C20312D323535203D3D20302E3173209A
:100440002D2035306D696E29002A2A2A2A2A2A2A67
:100450002A2A2A2A2A2A2A2A2A2A2A2A2A2A2A2AFC
:100460002A2A2A2A2A2A0052582041636B656420CE
:100470002D2072657665727420737563636573737E
:1004800066756C21002A2A2A2A2A2A2A2A2A2A2A36
:100490002A2A2A2A2A2A2A2A2A2A2A2A2A2A2A2ABC
:1004A0002A2A002A2A2A2A2A2A2A2A2A2A2A2A2AD6
:1004B0002A2A2A2A2A2A2A2A2A2A2A2A2A2A2A2A9C
:1004C0000052582041636B6564202D207570646173
:1004D0007465207375636365737366756C21002A98
:1004E0002A2A2A2A2A2A2A2A2A2A2A2A2A2A2A2A6C
:1004F0002A2A2A2A2A2A2A2A2A2A2A2A0056616CE1
:1005000069642063686F69636573206172653A206E
:100510005B315D2D5B31365D20286368616E6E65F1
:100520006C20312D31362900536574206F7574703D
:10053000757420666F7220706F727420005B585D56
:100540002061626F7274206368616E6765732061F9
:100550006E64206578697420525820636F6E6669F6
:1005600067005B535D207361766520736574746901
:100570006E677320746F205258005B525D20726565
:10058000766572742052582073657474696E67734F
:1005900020746F2064656661756C747300557365B3
:1005A000206E756D62657273205B312D445D207421
:1005B0006F206564697420706F727473205B452DC1
:1005C000515D20666F722073657474696E67730085
:1005D000202D20726563656976657220636F6E6693
:1005E0006967757261746F722C207278207377203E
:1005F000000A0A6F70656E4C52536E672000536597
:10060000742073657269616C2062617564726174D3
:10061000653A200056616C69642063686F696365A0
:10062000733A2031202D20342B34202F2032202DDE
:100630002038202F2033202D20382B34202F203419
:10064000202D203132202F2035202D2031322B3407
:10065000202F2036202D203136005365742043682A
:10066000616E6E656C20636F6E6669673A20005339
:1006700065742044617461726174652028302D3284
:10068000293A200053657420486F70206368616EBA
:100690006E656C7320286D61782032342C20736570
:1006A0007061726174656420627920636F6D6D6141
:1006B00073292076616C69642076616C756573209E
:1006C000312D3235353A2000536574206368616EF0
:1006D0006E656C2073706163696E672028783130B5
:1006E0006B487A293A200053657420524620706F77
:1006F0007765722028302D37293A20005365742001
:100700005246206D616769632028686578292065F5
:100710002E672E20307844454144463030443A20FC
:10072000005365742062617365206672657175653A
:100730006E63792028696E20487A293A20005B5A36
:100740005D20656E74657220726563656976657299
:1007500020636F6E66696775726174696F6E20756C
:1007600074696C79005B465D20646973706C6179B3
:100770002061637475616C206672657175656E6366
:100780006965732075736564005B525D2063616CFD
:1007900063756C6174652072616E646F6D206B654A
:1007A0007920616E6420686F70206C697374005BDF
:1007B000495D207265696E697469616C697A65204A
:1007C00073657474696E677320746F20736B6574DE
:1007D00063682064656661756C7473005B585D20A6
:1007E000726576657274206368616E6765732061F7
:1007F0006E642065786974206D656E75005B535D6D
:1008000020736176652073657474696E67732074F4
:100810006F20454550524F4D20616E6420657869C8
:1008200074206D656E7500557365206E756D62651B
:100830007273205B302D395D20746F20656469749C
:1008400020706172616D657465727300202D205394
:10085000797374656D20636F6E6669677572617414
:10086000696F6E000A0A6F70656E4C52536E672096
:10087000005129204F7574707574206265666F721F
:1008800065206C696E6B20283D465329203A200074
:10089000502920536C617665206D6F646520286552
:1008A00078706572696D656E74616C293A20004FCD
:1008B000292054696D65642042494E4420617420AA
:1008C0007374617274757020203A20004E29205094
:1008D000504D206F7574707574206C696D69746506
:1008E0006420202020203A200044495341424C45B6
:1008F00044004D292050504D205253534920746FCD
:10090000206368616E6E656C202020203A20004CC8
:10091000292050504D206D696E696D756D20737979
:100920006E63202875732920203A200044495341E2
:10093000424C4544004B29204661696C73616665F1
:1009400020626561636F6E20696E74762E20283197
:100950002D32353573293A20004A29204661696CC9
:100960007361666520626561636F6E2064656C61AA
:10097000792028302D323535203D3E20313073200E
:100980002D203135306D696E293A200049292046E5
:1009900061696C7361666520626561636F6E206674
:1009A00072712E203A200048292050574D20737430
:1009B0006F702064656C6179202020202020203A0F
:1009C000200047292050504D2073746F70206465BB
:1009D0006C6179202020202020203A200046292008
:1009E0004661696C736166652064656C617920207D
:1009F00020202020203A200050574D206368616E4F
:100A00006E656C200066756E6374696F6E3A2000C7
:100A10002920706F72742000506F776572546F7761
:100A2000657200445446205548462033322D626991
:100A3000742031306368004F70656E4C52536E679E
:100A40005258206D696E6920342F36636800466CF9
:100A50007974726F6E2F4F72616E676552582055B0
:100A600048462038636800525820747970653A20EF
:100A70000044697361626C656400487A00203D3D02
:100A8000200043616C63756C617465642070616300
:100A90006B657420696E74657276616C3A200042F1
:100AA00029204D6963726F202868616C6629205087
:100AB000504D202020203A00412920496E76657251
:100AC0007465642050504D20696E20202020203A0B
:100AD000003029204D7574652062757A7A65722020
:100AE000286D6F73746C79293A0039292053657227
:100AF00069616C2062617564726174653A00736D3E
:100B0000617274506F7274004672536B7900547244
:100B1000616E73706172656E740044697361626CBA
:100B200065640038292054656C656D657472793A86
:100B300020202020202020003729204368616E6E6D
:100B4000656C20636F6E6669673A20200036292045
:100B500044617461726174652028302D32293A2015
:100B6000202000352920486F70206368616E6E6513
:100B70006C733A2020202020003429204368616EC5
:100B80006E656C2073706163696E673A2020003374
:100B90002920524620706F7765722028302D372922
:100BA0003A202020003229205246206D6167696377
:100BB0003A202020202020202020003129204261BE
:100BC0007365206672657175656E63793A202020C1
:100BD0000000000000240027002A0000000000257B
:100BE0000028002B0000000000230026002900043C
:100BF00004040404040404020202020202030303C4
:100C000003030301020408102040800102040810BD
:100C1000200102040810200000000700020100006B
:100C20000304060000000000000000006E2E1124E6
:100C30001FBECFEFD8E0DEBFCDBF13E0A0E0B1E034
:100C4000EEE1FFE502C005900D92A639B107D9F794
:100C500016E0A6E9B3E001C01D92A734B107E1F7A1
:100C60001CE0CEE2DCE004C02297FE010E946A2F65
:100C7000CC32D107C9F70E94B32E0C948D2F0C945F
:100C80000000A0E0B0E0E7E4F6E00C94392FEC01BE
:100C9000A880B980CA80DB80A114B104C104D1044A
:100CA00041F484E2A82E89EDB82E8BE5C82E87E0AA
:100CB000D82EC601B5012DE133EF41E050E00E948E
:100CC000162F27EA31E440E050E00E94C22E7B015B
:100CD0008C01C601B5012DE133EF41E050E00E94E7
:100CE000162FCA01B9012CEE34EF4FEF5FEF0E94CF
:100CF000C22E6E0D7F1D801F911F97FF04C0615093
:100D0000704080409048688379838A839B839B01ED
:100D1000AC015F77B901CA01CDB7DEB7EAE00C9448
:100D2000552F0E944106089581EB92E00E944106F2
:100D300008956093B1027093B2028093B3029093CE
:100D4000B4020895A0E0B0E0E8EAF6E00C94322F97
:100D5000EC012B016A016115710519F0FB0191830A
:100D60008083C114D10449F0C6010297839728F00B
:100D700020E030E040E050E0DCC0A9908A2D90E017
:100D80000E94822F892BC9F7FDE2AF1621F4A990AA
:100D90003324339405C08BE2A81609F4A9903324B8
:100DA000C114D10421F0E0E1CE16D10411F5F0E335
:100DB000AF1669F48881883711F0883541F4A9802D
:100DC000229682E0382A20E1C22ED12C12C0C11412
:100DD000D10479F4E0E3AE1659F199E9E92E99E9E5
:100DE000F92E99E9092F99E1192F8AE0C82ED12C03
:100DF0003AC0FAE0CF16D10491F080E1C816D104D0
:100E000029F0E8E0CE16D104F9F415C0BFEFEB2EBF
:100E1000BFEFFB2EBFEF0B2FBFE01B2F24C0A9E9B4
:100E2000EA2EA9E9FA2EA9E90A2FA9E11A2F1BC077
:100E3000F8E0CF2ED12CEFEFEE2EEFEFFE2EEFEFFE
:100E40000E2FEFE11E2F0FC09601442737FD40956E
:100E5000542F6FEF7FEF8FEF9FEF0E94F42EC901A9
:100E6000DA017C018D0120E030E040E050E060E0FC
:100E70003601882477FC8094982C70EDB72EBA0C3C
:100E8000F9E0FB1570F48A2D81548A3118F499EC3D
:100E9000B92E06C08A2D81568A3148F589EAB82EC6
:100EA000BA0C8B2D90E08C159D050CF56F3FE9F089
:100EB000E216F30604071507B8F0CA01B901A40148
:100EC00093010E94C22E9B01AC018B2D90E0A0E00B
:100ED000B0E0280F391F4A1F5B1F281739074A0740
:100EE0005B0710F061E001C06FEFA990C6CF41141D
:100EF000510451F0662311F0219703C031FE04C064
:100F00002297F201D183C08330FE07C050954095EF
:100F1000309521953F4F4F4F5F4F67FF0AC082E2E8
:100F200090E090934606809345062FEF3FEF4FEFFA
:100F30005FEFB901CA01CDB7DEB7E1E10C944E2FE6
:100F4000FC0188279927E89421912032E9F3293080
:100F500010F02E30C8F32B3241F02D3239F4689462
:100F600004C00E94F507820F911D219120532A3061
:100F7000C0F31EF4909581959F4F089546E953E084
:100F80000E94C3070895009731F4DA018D919C9176
:100F9000009709F40EC0DC01FB013D912191222351
:100FA00019F03217C9F3FACF332331F4DA011D9265
:100FB0001C928827992708951197AF93BF93FB013F
:100FC0003D912191321771F4332321F48827992719
:100FD000119702C01E921196FA01A193B0839F91BE
:100FE0008F910895222369F7EACF7AE0979F902D99
:100FF000879F802D910D1124089580919803813051
:1010000019F482E08093980380919803833019F457
:1010100084E0809398030895E3E0F0E089E0809312
:101020005700849190E08670863009F491E0892F12
:1010300008951F93182F0E940C08882379F09FB7FA
:1010400081E080938D05F894A89588E180936000F5
:1010500010936000112309F0A8959FBF1F91089578
:10106000382F20E080911F0590912005822793273B
:1010700040E061E270E19C01220F331F97FF04C042
:10108000C9018627972701C0C9014F5F483099F7EA
:101090009093200580931F05089586E38093BE03F7
:1010A00080E092ECA1E0B0E08093BF039093C00396
:1010B000A093C103B093C20387E08093CB0380EC7D
:1010C00092E9ADEEB9E18093C3039093C403A0937A
:1010D000C503B093C60385E08093CC038DEE9EEFED
:1010E000ADEABEED8093C7039093C803A093C903F4
:1010F000B093CA03ADECB3E080E090E0863010F02E
:10110000E0E004C0FC01E058FC4FE081ED93019663
:101110008831910599F782E08093E5038AE0809316
:10112000E603089580EC91EDA8E9BBE180939B0371
:1011300090939C03A0939D03B0939E0310929F03F2
:101140001092A0031092A1031092A2030895843676
:10115000910520F4BC0180E090E025C08E3B910514
:1011600050F48A559040BC0180E090E02AE030E0E5
:1011700040E050E016C0823D910550F4845B904001
:10118000BC0180E090E024E630E040E050E009C09F
:101190008D5C9040BC0180E090E028E532E040E0CA
:1011A00050E00E94C22E24E630E040E050E00E9471
:1011B000C22E089590E08C599F4F0E94A708089571
:1011C000DC019896EC91F0E0E770F070E858FC4F85
:1011D000808108958F929F92AF92BF92CF92DF92BB
:1011E000EF92FF920F931F938C010E94E008D801A9
:1011F00097962C9130E043E150E0249FF001259F29
:10120000F00D349FF00D1124EB54FD4F8080918040
:10121000A280B38090E00F96AA2797FDA095BA2FE1
:10122000BC01CD0120E43FE14DE750E00E94C22E19
:10123000A50194010E94F42E69017A0180ED97E0E6
:10124000A0E0B0E0C80ED91EEA1EFB1ED801989699
:101250008C91887181F060E07EEE8AEB9BE0A501C5
:1012600094010E94F42E28513C4F4F4F5F4FC20E05
:10127000D31EE41EF51E87EE93E0A0E0B0E0C80E9A
:10128000D91EEA1EFB1EC701B60128EE33E040E07E
:1012900050E00E94F42ECA01B90128EE33E040E08C
:1012A00050E00E94C22E1F910F91FF90EF90DF90AF
:1012B000CF90BF90AF909F908F9008958F3F9105F2
:1012C00009F010F480E0089522E08030920710F4D5
:1012D00081E008958050934010F083E0089582E00B
:1012E0000895CF92DF92FF920F931F93CF93DF93D6
:1012F000F82FEB016A01182F1695E0E0888199819B
:10130000D6018C938A819B8111968C9311978C8145
:101310009D8112968C9312978E819F8113968C9348
:101320001397288139814A815B816C817D818E810F
:101330009F819295990F990F907C832F8370982BA2
:10134000852F8370880F880F982B872F8370829545
:10135000807F982B14969C9385E090E0C80ED91E50
:101360002896EF5F1E1750F6F0FF21C08881998103
:101370000E945E09F82E8A819B810E945E09182FC7
:101380008C819D810E945E09082F8E819F810E9421
:101390005E09F294FF0CFF0C70ECF7221295107F9F
:1013A0001F29182B000F000F012BD6010C93DF9182
:1013B000CF911F910F91FF90DF90CF90089523E080
:1013C0008032920718F420E030E026C023E0883E07
:1013D000920748F49C012F51334054E036952795ED
:1013E0005A95E1F719C027E0803D920720F49C014F
:1013F0002C5D334011C028E08839920718F02FEF98
:1014000033E00AC09C01285C374044E036952795BC
:101410004A95E1F72D503C4FC90108958C30910554
:1014200048F49C0174E0220F331F7A95E1F7285DA0
:101430003C4F17C023E0843F920720F49C012452C4
:101440003C4F0FC024E08030920718F020E938E0CC
:1014500008C09C012657334F64E0220F331F6A9562
:10146000E1F7C90108959C013695279525753575D5
:10147000821B930B9C0136952795369527952373F0
:10148000337383739373280F391FC901E4E0969572
:101490008795EA95E1F7820F931F8F709F7021E087
:1014A00031E0AC01429FC001439F900D529F900DCF
:1014B0001124892F0895882339F05F980000289A15
:1014C00000005F9A000008955F98000028980000CF
:1014D0005F9A000008955F9A000083B15F98000052
:1014E00090E096958795817008950F931F93082F2C
:1014F0005C9A5F985C9810E0802F80780E945B0A6D
:10150000000F1F5F1830C1F75F981F910F9108956A
:101510008F770E94750A08950F931F93082F10E08C
:10152000802F80780E945B0A000F1F5F1830C1F780
:101530005F981F910F9108950F931F935F9880E01C
:1015400000E0182F110F0E946B0A810F0F5F083007
:10155000C1F71F910F9108950E94880A0E949C0A6A
:101560005C9A08951F93162F80680E94750A812F38
:101570000E948C0A5C9A1F9108951F931091C703D3
:101580001827EEEBF3E0E80FF11D89E767850E946D
:10159000B20A8DE3612F0E94B20A82E4612F0E9499
:1015A000B20A1F91089586E20E94AC0A08950F9333
:1015B0001F938C018CE1F80164810E94B20A8DE1D5
:1015C000F80165810E94B20A8EE1F80166810E94ED
:1015D000B20A80E2F80167810E94B20A81E2F80152
:1015E00060850E94B20A82E2F80161850E94B20A17
:1015F00083E2F80162850E94B20A84E2F801638501
:101600000E94B20A85E2F80164850E94B20A8AE269
:10161000F80165850E94B20A8EE6F80166850E948F
:10162000B20A8FE6F80167850E94B20A80E7F801E6
:1016300060890E94B20A81E7F80161890E94B20ABA
:1016400082E7F80162890E94B20A1F910F91089502
:10165000EF92FF920F931F93CF93DF937B018C0147
:10166000603028E372072CE982072CE1920728F505
:1016700020E836E948E950E00E94F42EE901689735
:10168000B90180E090E020E839E647E65FEF0E948C
:10169000C22E6E0D7F1D801F911F32E0660F771FD7
:1016A000881F991F3A95D1F721E732E040E050E0DA
:1016B0000E94F42E890180E421C020E03DE241E354
:1016C00051E00E94F42EE9016897B90180E090E0B2
:1016D00020E033ED4EEC5EEF0E94C22E6E0D7F1DBA
:1016E000801F911F660F771F881F991F21E732E027
:1016F00040E050E00E94F42E890180E69E012F71A7
:10170000622F680F85E70E94B20A86E7612F0E9468
:10171000B20A87E7602F0E94B20ACDB7DEB7E6E0D3
:101720000C94592F9F92AF92BF92CF92DF920F935A
:10173000DF93CF9300D000D0CDB7DEB7982E83E0F3
:101740000E94AC0A8093E70384E00E94AC0A809375
:10175000E80386E060E00E94B20A87E061E00E9450
:10176000B20A89E06FE70E94B20A8AE065E00E944F
:10177000B20A8BE062E10E94B20A8CE065E10E944D
:10178000B20A8DE06DEF0E94B20A8EE060E00E9426
:10179000B20A992019F084E193E008C08091E50332
:1017A00023E1829FC00111248B549D4F0E94D70AD0
:1017B00080E36CE80E94B20A82E36FE00E94B20A02
:1017C00083E362E40E94B20A84E36AE00E94B20A00
:1017D00085E36AE20E94B20A86E36DE20E94B20AE1
:1017E00087E364ED0E94B20A88E360E00E94B20AD7
:1017F00089E360E00E94B20A992049F065E7A62ECD
:1018000061ECB62E61ECC62E6EEDD62E08C0A0900F
:10181000C703B090C803C090C903D090CA030AE3BD
:101820008D2D9927AA27BB2789839A83AB83BC83F5
:10183000802F69810E94B20A802F8B5F69810E948C
:10184000B20ADC2CCB2CBA2CAA240F5F0E3341F742
:1018500083E46FEF0E94B20A84E46FEF0E94B20A41
:1018600085E46FEF0E94B20A86E46FEF0E94B20A2D
:10187000992019F08DE666E003C08DE66091CB03F8
:101880000E94B20A89E760E00E94B20A8AE760918A
:10189000CC030E94B20A83E760E00E94B20A84E7A8
:1018A00060E00E94B20A992029F060EC72E98DEEA6
:1018B00099E108C06091C3037091C4038091C5038E
:1018C0009091C6030E94280B0F900F900F900F90DD
:1018D000CF91DF910F91DF90CF90BF90AF909F900D
:1018E000089587E061E00E94B20A8EE764E20E94F8
:1018F000B20A88E063E00E94B20A88E060E00E94D9
:10190000B20A87E065E00E94B20A85E062E00E94C8
:10191000B20A83E00E94AC0A8093E70384E00E944D
:10192000AC0A8093E8030895582F40918C04842FCB
:1019300090E0FC01EF70F0709F012F5F3F4F74E06B
:10194000959587957A95E1F72817390751F0E4586E
:10195000FB4F5083842F8F5F8F70407F842B809349
:101960008C0408951F920F920FB60F921124EF92DC
:10197000FF920F931F932F933F934F935F936F9318
:101980007F938F939F93AF93BF93EF93FF93E090D9
:101990009F03F090A0030091A1031091A20389B1CD
:1019A000A8019701207430704070507090E003E0FF
:1019B000969587950A95E1F7A0E0B0E08170907068
:1019C000A070B070281739074A075B0709F452C0A6
:1019D000209184003091850010928500109284003F
:1019E0008091AD04882309F045C0E5FC02C036951E
:1019F000279589E0253C380708F180914703863018
:101A0000D0F0809147038F3FB1F020E00EC0E22F6D
:101A1000F0E0EE0FFF1FDF01A255BB4F8D919C91AF
:101A2000E95DFC4F918380832F5F809147032817E6
:101A300070F31092AC04109247031CC082E02D3B5F
:101A40003807A8F080914703803188F4109147034C
:101A5000C9010E94DF09E12FF0E0EE0FFF1FE25500
:101A6000FB4F918380831F5F1093470303C08FEF69
:101A700080934703FF91EF91BF91AF919F918F9119
:101A80007F916F915F914F913F912F911F910F9196
:101A9000FF90EF900F900FBE0F901F90189583E06E
:101AA000809380008AE1809381008FEF9FEF909375
:101AB00089008093880010926F0088E080936D0009
:101AC000E8E6F0E080818460808308956F3020F044
:101AD00086958695805408958DE0689F802D112409
:101AE0000895882319F460E071E002C063E071E0BA
:101AF00083E296E00E94762C0895A0E0B0E0E3E84F
:101B0000FDE00C943B2F182F0E9449299B01AC014A
:101B10008091190590911A05A0911B05B0911C05A3
:101B200069017A01C81AD90AEA0AFB0AD701C60173
:101B300089589341A040B04010F0109218052093AE
:101B4000190530931A0540931B0550931C052091ED
:101B5000AD04822F81508230E8F5809118058823EA
:101B600009F44FC1813011F482E0BCC1803108F02A
:101B700035C1E82FF0E0E255FB4F10838F5F809373
:101B80001805803109F0B0C1A0EBB4E0213039F480
:101B90001196EC911197E695E6958C9109C08D917F
:101BA0009C911197E92FE695E695E6959695879590
:101BB000E03140F4F0E090E0EE0FFF1FE95DFC4FF4
:101BC000918380831092AC04129684E0AE3BB807F8
:101BD000E9F68AC1233009F004C1809118058823F1
:101BE00021F41F3009F080C10CC1883130F4E82F96
:101BF000F0E0E355FB4F108374C1883109F0EEC06B
:101C0000112309F0EBC0C0E0D0E00BE010E0DE01F2
:101C100063E0AA0FBB1F6A95E1F7C09FB001C19FA7
:101C2000700DD09F700D1124FB01E255FB4F808198
:101C30002181922F977095958795FD01EE0FFF1FDB
:101C4000E95DFC4F91838083FB01E155FB4F3081BF
:101C50003695369536952181422F4295440F407E28
:101C6000842F832B269526952695922F97709595F0
:101C70008795FD01EE0FFF1FE75DFC4F9183808389
:101C8000FB01E055FB4F8081829586958695837098
:101C90004181942F990F990F292F282B4295469512
:101CA0004695437082818170880F880F382F342BBE
:101CB00035952795FD01EE0FFF1FE55DFC4F318344
:101CC0002083FB01EE54FB4F308136952181422F5A
:101CD000479544274795842F832B2695922F9770FD
:101CE00095958795FD01EE0FFF1FE35DFC4F9183F6
:101CF0008083FB01ED54FB4F308132953F70218191
:101D0000422F4295407F842F832B22952F70922F54
:101D1000977095958795FD01EE0FFF1FE15DFC4FD4
:101D200091838083FB01EC54FB4F8081881F8827BF
:101D3000881F4181942F990F292F282B441F442756
:101D4000441F82818370880F382F342B3595279557
:101D5000FD01EE0FFF1FEF5CFC4F31832083FB0181
:101D6000EA54FB4F3081369536952181422F4295BA
:101D7000440F440F407C842F832B26952695922F69
:101D8000977095958795AA0FBB1FFD01ED5CFC4FE1
:101D90009183808369547B4FFB0120812295269596
:101DA00027704181342F330F330F330F832F822B52
:101DB000942F92959695977095958795AB5CBC4FAF
:101DC00011969C938E932196C230D10509F01FCFB6
:101DD0008091C40483FD02C01092AC0410921805D7
:101DE00083C0243009F080C040911805442359F481
:101DF000183AB1F41092200510921F0588EA0E944B
:101E0000300881E06FC0413019F410931D0504C003
:101E1000423031F410931E05812F0E9430085DC0BE
:101E200060911E05262F30E0220F331FE42FF0E0D3
:101E3000C90102968E179F0734F0433268F7E555C3
:101E4000FB4F1083E9CF2D5F3F4F40911F0550910D
:101E50002005E217F30749F4912F80E0482759271E
:101E60005093200540931F0538C0812F90E04817FC
:101E7000590789F580911D05813069F5613118F0A8
:101E800080E180931E05D0901E054EEAE42E44E0CA
:101E9000F42E00E010E01BC0F701D081C0E081818A
:101EA00090E08C2B9D2B33E0969587953A95E1F742
:101EB0000E94DF09F801EE0FFF1FE95DFC4F9183DF
:101EC00080830F5F1F4F82E090E0E80EF91E0D1532
:101ED00018F31092AC04109218058091180588230D
:101EE00019F08F5F80931805CDB7DEB7E8E00C944A
:101EF000572FFF920F931F93CF93DF93182F092F24
:101F0000F62E8EE30E94B20A212F302FC901EC0178
:101F100010E005C08FE769910E94B20A1F5F1F158C
:101F2000C8F385E064E00E94B20A83E00E94AC0A34
:101F30008093E70384E00E94AC0A8093E8030E9448
:101F400049296093E9037093EA038093EB0390932C
:101F5000EC0387E069E00E94B20A81E08093980375
:101F6000CDB7DEB7E5E00C945A2F0E94790F80912F
:101F700098038130D9F40E9449292091E9033091D6
:101F8000EA034091EB035091EC03621B730B840B4B
:101F9000950B605A76488140904040F4E8CF83E248
:101FA00096E067E071E00E94762C08958091980396
:101FB0008130A9F3089583E296E06EE70E942E2E09
:101FC0000895A0E0B0E0E7EEFFE00C943A2F6C013A
:101FD00083E296E06EE70E942E2E760100E010E08C
:101FE000C0E0D0E0B0E2BB2E0AC00830110521F4F9
:101FF0009E012095F60120870894E11CF11CF70151
:102000006081862F8D57823040F483E296E06DE741
:102010000E942E2EF70160816B2583E296E00E94DC
:102020002E2E0115110551F0F70180819E01280F18
:10203000311DC32FDD27C20FD31FD0700F5F1F4F7D
:102040000930110591F6CDB7DEB7E9E00C94562FB3
:10205000A9E0B0E0EEE2F0E10C94412F382FE62F3A
:102060008091910490E0019664E270E00E94E12E7C
:10207000982F8093910488E9898380E18A83913045
:1020800071F0913028F0923099F09330E1F416C05D
:1020900085E08B8381EF8C832F5F2D8317C09B831B
:1020A00081EF8C8384E6489FC00111249D830EC07C
:1020B00084E08B8381EF8C833D8308C09B8381EF19
:1020C0008C83ED8303C00E94DB0F04C0CE01019618
:1020D0000E94E10F2996E2E00C945D2F0F931F936D
:1020E000CF93DF93182F092F83E296E06EE70E94CB
:1020F0002E2E212F302FC901EC0110E000E2888143
:102100008D57823040F483E296E06DE70E942E2ED8
:1021100088818027888383E296E069910E942E2E31
:102120001F5F193061F783E296E06EE70E942E2E62
:10213000DF91CF911F910F910895A9E0B0E0E3EAFC
:10214000F0E10C94412F382F80919104882379F489
:102150008EEF89833A836B83842F90E095958795E2
:102160008C832D83198618861F821E822FC0409172
:102170008C04842F90E09C012F70307054E0959572
:1021800087955A95E1F78217930721F18DEF89839F
:102190001A821B82DE01149620E008C0E458FB4F2F
:1021A00080818D93405F2F5F263069F0842F90E00F
:1021B000FC0134E0F595E7953A95E1F78F70907062
:1021C000E817F90759F740938C042A83CE0101964A
:1021D0000E946E108091910490E0019666E070E09C
:1021E0000E94E12E809391042996E2E00C945D2FE9
:1021F0009F92AF92BF92CF92DF92EF92FF920F9396
:102200001F93B82EA62ED42EC22E902E0E9449299E
:102210007B018C0180917B0420918D0430918E0490
:1022200040918F04509190048823B1F0D801C701E8
:10223000821B930BA40BB50B815E9E42A040B04065
:1022400020F12C2DDC1408F42D2D8B2D6A2D422F1E
:10225000292D0E94281011C0D801C701821B930BA1
:10226000A40BB50B81539547A040B04070F08B2D67
:102270006A2D4D2D2C2D0E949D10E0928D04F09220
:102280008E0400938F04109390041F910F91FF9080
:10229000EF90DF90CF90BF90AF909F90089583E232
:1022A00096E06091EE030E942E2E08951F93182F42
:1022B00083E296E0612F0E942E2E8091EE0381270B
:1022C0008093EE031F9108951F93192F0E945611BA
:1022D000812F0E9456111F910895DF92EF92FF9275
:1022E0000F931F93D82E7B011092EE0303E216E0AA
:1022F000C80165EB0E942E2EC80162E60E942E2EB8
:102300008D2D0E945611C7010E9464111F910F91DB
:10231000FF90EF90DF90089589E060E00E94CE2961
:1023200088E061E00E94CE2987E061E00E94CE292A
:1023300082E060E00E94CE2984E061E00E94CE2924
:102340000895892B19F08AE061E002C08AE060E01C
:102350000E943A2A0895A0E0B0E0E1EBF1E10C948C
:10236000392F8CE00E94AC0A882379F583E296E04D
:1023700063E171E00E94762C2D9A80E00E94920B1E
:102380000E94710C2D9821C083E296E00E94F52DE9
:10239000482F8091AD04882321F0842F0E947D0D69
:1023A00014C080911605E82FF0E031969F012F713F
:1023B000307031978091150590E02817390729F082
:1023C000E451FB4F40832093160583E296E00E9480
:1023D000BB2D892BC9F680919803843009F08CC0FD
:1023E0000E94492960939C0470939D0480939E04ED
:1023F00090939F04611571058105910561F481E059
:1024000090E0A0E0B0E080939C0490939D04A093A2
:102410009E04B0939F048091A8049091A9048160C8
:102420009093A9048093A80483E0809398038FE796
:102430000E94880AC3EED4E00E949C0A899304E0BB
:10244000CC3ED007C9F74091CE048091E304282FF9
:1024500030E0842F90E08227932786FF40C080E4FD
:1024600048274093CE04C90188739070C89709F536
:1024700010E014C01F5F8091E603E12FF0E084FFBD
:1024800006C0ED51FB4F80810E94940C07C0ED51B6
:10249000FB4F83E296E060810E942E2E212F30E0D8
:1024A0008091E30490E0877090708217930714F78F
:1024B00016C02F733070232B91F48091E404809325
:1024C000A0048091E5048093A2048091E6048093A7
:1024D000A3048091E9048093AA041092AB04809134
:1024E0001705813019F482E0809317058091170554
:1024F000833011F4109217050E9449295B016C0189
:102500008091A4049091A504A091A604B091A70481
:102510000097A105B105C9F0A6019501281B390B4B
:102520004A0B5B0BDA01C901885B9B40A040B040BD
:1025300060F00E94D30A8093A1041092A404109228
:10254000A5041092A6041092A7048EEB93E00E94BB
:10255000EA08209198043091990440919A0450918E
:102560009B0486017501E21AF30A040B150BE616AB
:10257000F7060807190708F4EAC0A0929804B09279
:102580009904C0929A04D0929B04A8958091AC04BF
:10259000883008F0D4C08091AC048F5F8093AC0485
:1025A000E0909C04F0909D0400919E0410919F0483
:1025B000E114F1040105110511F18EEB93E00E9485
:1025C000EA08AE18BF08C00AD10A6A157B058C0557
:1025D0009D0588F480919F0384FD04C080ED97E001
:1025E0000E94A11110929C0410929D0410929E04CE
:1025F00010929F0404C080E090E00E94A11190918D
:10260000CE04907C9093CE04009116051091150590
:102610000117B1F180911705823091F59058909390
:10262000CE048EEB93E00E94E008893010F048E081
:1026300002C0482F415030E013C03F5FA32FB0E0ED
:10264000812F90E0FC01E451FB4F2081FD01E2531A
:10265000FB4F2083A45FBA4F2C930196182F1F7154
:10266000341710F4101749F710931505832F895C60
:102670009091CE04892B8093CE0430930C051AC020
:10268000209117052430D1F490910C05EDE0F5E090
:10269000AFECB4E0292F30E02E0F3F1F02C0819134
:1026A0008D93E217F307D9F7995C8091CE04982BAC
:1026B0009093CE0483E08093170523C08091930408
:1026C000823029F491609093CE042D9A0FC090939C
:1026D000CE042D98222319F481E080931705809170
:1026E0001705833019F484E080931705F8948091DE
:1026F000E603877067E273E04FEC54E00E947109D3
:1027000078942C9A809192040E94BD0A8EEB93E0FB
:102710000E94E008682F8EEC94E00E94790FE0910F
:102720009204EF5FE0939204E83131F0F0E0E2547C
:10273000FC4F8785882359F41092920408C0809139
:10274000AC04883009F42D9A89E08093AC04809120
:10275000E603887171F180919803823051F5809180
:10276000A8049091A904880F991F9093A9048093BD
:10277000A80483E0809398030E94710C0E94492969
:102780006093A4047093A5048093A6049093A70477
:10279000611571058105910561F481E090E0A0E08B
:1027A000B0E08093A4049093A504A093A604B093F2
:1027B000A7048091E60384FF1EC08091A804909135
:1027C000A9048E7F0E94330A182F8091A004609183
:1027D000AA040E94660D082F8091A104612F0E9417
:1027E000660D282F8091A2046091A304402F0091D0
:1027F00099030E94F8102C98809193048130C9F0BD
:10280000813020F0823009F03FC033C08BE00E945D
:102810006D2A892BC9F581E0809393040E943B299E
:102820006093940470939504809396049093970416
:102830002BC08BE00E946D2A892B21F50E943B2939
:1028400020919404309195044091960450919704FE
:10285000621B730B840B950B695E73408040904044
:1028600098F082E08093930480ED97E00E94A1119C
:102870000BC08BE00E946D2A892B31F080E090E044
:102880000E94A11110929304CDB7DEB7EAE00C9438
:10289000552F8AE061E00E94CE298AE060E00E9424
:1028A0003A2A08951F93182F0E94492960938D0496
:1028B00070938E0480938F049093900410937B0404
:1028C000112329F440E855E260E070E004C040E0E4
:1028D00051EE60E070E083E296E00E94342D1F919B
:1028E0000895ACE1B0E0E7E7F4E10C94392F0E94E1
:1028F00049297B018C0181E00E94920BA4E7AA2E5A
:102900006E010894C11CD11CF3E0BF2EA982C60140
:1029100061E00E94B50FB09298030E94710C6AEFBB
:1029200070E080E090E00E946F29809198038330EE
:1029300009F07DC083E296E00E94BB2D892B09F04F
:1029400076C00E9449296E197F09800B910B60584F
:10295000734C894C914008F06AC0D8CF8FE70E9431
:10296000880A0E949C0A843509F05CC089830E9411
:102970009C0A182F00E010937A04009379040E94B7
:102980009C0A080F111D10937A04009379040E9489
:102990009C0A809378040E949C0A8093770481317A
:1029A00008F040C0FF2407C00E949C0A095A1B4F30
:1029B000F8018083F3940F2D10E08091770490E06C
:1029C000880F991F0817190778F380E78983CE01CC
:1029D000019661E00E94B50F83E0809398030E9406
:1029E000710C62E370E080E090E00E946F298091BA
:1029F00098038330A9F08FE70E94880A0E949C0AFE
:102A0000803581F4898303EA13E00E949C0AF8016F
:102A100081938F01F3E00E3B1F07B9F781E003C0FC
:102A200082E001C083E06C96EAE00C94552F80911F
:102A30009803833009F092CFF3CF83E00E94AC0A71
:102A40008093E70384E00E94AC0A8093E80387E068
:102A500061E00E94B20A6AE070E080E090E00E94CB
:102A60006F290E94710C000008950F931F93082F87
:102A700017C02D9A64E670E080E090E00E946F2914
:102A80002D9864E670E080E090E00E946F291F5F5F
:102A9000101778F36CE271E080E090E00E946F29FB
:102AA00010E0F6CF482F392F25E00DC0F999FECF61
:102AB0001FBA842F932F92BD81BD60BD0FB6F894CD
:102AC000FA9AF99A0FBE215059F0F999FECF842F46
:102AD000932F92BD81BDF89A80B5681739F7089594
:102AE00082E00E9435150895A0E0B0E0EAE7F5E144
:102AF0000C94322F482E562EEE24FF24882499243D
:102B0000C0E0D0E0CC24DD2436E3332E04C05524CD
:102B10005394CC24DD24442069F480919903839D4F
:102B2000E00111242AE9E22E23E0F22E99E0892E19
:102B3000912C1DC021E0421671F480919903839D70
:102B4000E00111242B968EEBE82E83E0F82E09E2AB
:102B5000802E912C0CC032E0431649F419E9E12E85
:102B600013E0F12EB1E08B2E912CC8EDD0E03E01A8
:102B70006C0C7D1C1092200510921F05E3011BC0F8
:102B8000552059F4F999FECFD2BDC1BDF89A80B550
:102B9000F701E00FF11F808307C0F701E00FF11F7D
:102BA000CE0160810E9452150E0D1F1DF80180811B
:102BB0000E94300821969E012619022F10E0081568
:102BC0001905F0F2CE015520D9F4F999FECFD2BD06
:102BD000C1BDF89A20B5F999FECF2196D2BDC1BDED
:102BE0002197F89A80B590E0B22EAA248A299B29D1
:102BF00020911F05309120052817390759F487CFF8
:102C00002196609120050E945215CE0160911F050A
:102C10000E94521580E091E0C80ED91E91E0C916BD
:102C200093E0D90608F477CF852DCDB7DEB7E1E183
:102C30000C944E2F80E061E00E94741581E061E009
:102C40000E947415089580E060E00E947415882346
:102C500031F081E060E00E947415882331F40E9415
:102C600092080E944D080E941A16089582E061E0C1
:102C70000E947415089582E060E00E9474158091AE
:102C80009903843020F0109299030E94361608951B
:102C90001F93182F0E943B1680919903811731F0E2
:102CA000143020F4109399030E9436161F91089552
:102CB0001092550485E6E0EFF3E0DF011D928A955E
:102CC000E9F708951F93182F8F3711F08830E1F539
:102CD000E0915504EE2309F455C0E150E09355040A
:102CE000F0E0E051FC4F108283E296E06DE00E943C
:102CF0002E2E10E00AC0E12FF0E0E051FC4F83E2FD
:102D000096E060810E942E2E1F5F80915504181757
:102D100090F383E296E060E20E942E2E83E296E03A
:102D20006DE00E942E2E10E00AC0E12FF0E0E0518D
:102D3000FC4F83E296E060810E942E2E1F5F8091FF
:102D40005504181790F31CC08B3119F40E945816C3
:102D50001FC08D30E9F08A30D9F080915504843657
:102D600088F483E296E0612F0E942E2E8091550414
:102D7000E82FF0E0E051FC4F10838F5F8093550403
:102D800080E007C083E296E067E00E94E22AF8CF85
:102D900081E01F9108951F93CF93DF93CDECD3E093
:102DA00010E03BC083E296E062E271E00E94732C87
:102DB00083E296E0612F4AE050E00E94F02B83E22C
:102DC00096E06FE271E00E94732C699170E080E000
:102DD00090E02091CC0330E040E050E00E94C22E11
:102DE00020E137E240E050E00E94C22EDC01CB013E
:102DF0004091C3035091C4036091C5037091C60311
:102E0000480F591F6A1F7B1F83E296E02AE030E0DB
:102E10000E94B72B1F5F183119F08881882311F6A3
:102E2000DF91CF911F910895EF92FF920F931F931F
:102E3000882339F483E296E061E77AE00E94002B70
:102E40003BC090E00E94A70824E630E040E050E05C
:102E50000E94F42E122F032FF42EE52E622F732FD3
:102E6000842F952F2AE030E040E050E00E94F42EBD
:102E700083E296E0BA01A9012AE030E00E94A82B83
:102E800083E296E06EE20E94E22A612F702F8F2D7E
:102E90009E2D2AE030E040E050E00E94F42EAB018D
:102EA000BC0183E296E02AE030E00E94A82B83E296
:102EB00096E063E70E94142B1F910F91FF90EF9013
:102EC0000895FF920F931F93CF93DF9383E296E0D1
:102ED00067E67AE00E94C12A8091A303813041F421
:102EE00083E296E06EE47AE00E94002BFF246DC03E
:102EF000823029F483E296E067E37AE0F5CF84300C
:102F000029F483E296E063E27AE0EECF853071F750
:102F100083E296E068E17AE0E7CFCF2DD0E0C930D8
:102F2000D1051CF06F2D685C02C06F2D6F5C83E2D1
:102F300096E00E94E22A83E296E060E17AE00E9455
:102F4000C12ABE016F5F7F4F83E296E04AE050E006
:102F50000E944C2C83E296E065E07AE00E94C12A50
:102F60008E010D551C4FD8011196EC91E032F8F40A
:102F700083E296E068EF79E00E94C12AF80181813E
:102F8000803130F083E296E063E371E00E94732CBD
:102F9000CD55DC4F698170E06F7070706F5F7F4F4F
:102FA00083E296E04AE050E00E945F2C0DC0F0E022
:102FB000EF70F070EE0FFF1FE85BFC4F60817181D6
:102FC00083E296E00E94762CF39480917804F816C0
:102FD00008F4A3CF83E296E06DED79E00E94C12A68
:102FE0008091BB030E94141783E296E062EC79E0C3
:102FF0000E94C12A8091BC030E94141783E296E0CC
:1030000067EA79E00E94C12A8091BD030E941417EB
:1030100083E296E06CE879E00E94C12A4091B30314
:103020005091B4036091B5037091B60341155105F9
:103030006105710539F183E296E02AE030E00E94F3
:10304000B72B83E296E069E579E00E94C12A80917E
:10305000B7030E94DA08AB01BC0183E296E02AE0E4
:1030600030E00E94B72B83E296E065E379E00E94AE
:10307000C12A83E296E06091B8034AE050E00E94E2
:10308000022C06C083E296E06CE279E00E94002BFD
:1030900083E296E06FE079E00E94C12A6091B90373
:1030A0007091BA0383E296E04AE050E00E94DC2B84
:1030B00083E296E062EF78E00E94C12A6091B20359
:1030C000603150F470E06F5F7F4F83E296E04AE03A
:1030D00050E00E945F2C06C083E296E069EE78E043
:1030E0000E94002B83E296E06CEC78E00E94C12AFB
:1030F0008091B10380FD03C065E371E002C069E324
:1031000071E083E296E00E94762C83E296E06FEA1B
:1031100078E00E94C12A8091B10382700E94710DF3
:1031200083E296E060E978E00E94C12A8091B103D1
:1031300084700E94710D83E296E061E778E00E945E
:10314000C12A8091B10388700E94710DCDB7DEB79E
:10315000E5E00C945A2F1F93CF93DF9383E296E020
:103160006BEB7BE00E94C12A4091C3035091C403E2
:103170006091C5037091C60383E296E02AE030E0D7
:103180000E94B72B83E296E065EA7BE00E94C12AA9
:103190004091C7035091C8036091C9037091CA035D
:1031A00083E296E020E130E00E94B72B83E296E0D4
:1031B0006FE87BE00E94C12A83E296E06091CB0336
:1031C0004AE050E00E94022C83E296E069E77BE04F
:1031D0000E94C12A83E296E06091CC034AE050E06D
:1031E0000E94022C83E296E063E67BE00E94C12A03
:1031F000CDECD3E010E012C0112331F083E296E071
:103200006DE371E00E94732C83E296E069914AE0DD
:1032100050E00E94F02B1F5F183119F0888188233D
:1032200059F783E296E00E94EA2A83E296E06DE491
:103230007BE00E94C12A83E296E06091E5034AE0C8
:1032400050E00E94022C83E296E068E37BE00E945B
:10325000C12AE091E603F0E0E770F070EE0FFF1F87
:10326000E859FC4F6081718183E296E00E94762CE0
:1032700083E296E063E27BE00E94C12A8091E6034C
:1032800090E0887190708830910589F089309105BF
:103290001CF4892B39F01BC08031910569F04897E7
:1032A000B1F40FC083E296E06AE17BE00EC083E2F6
:1032B00096E06EE07BE009C083E296E068E07BE0A8
:1032C00004C083E296E06EEF7AE00E94002B83E276
:1032D00096E06AEE7AE00E94C12A4091BF035091C5
:1032E000C0036091C1037091C20383E296E02AE0BB
:1032F00030E00E94B72B83E296E061ED7AE00E9415
:10330000C12A80919F0380710E94710D83E296E033
:1033100068EB7AE00E94C12A80919F0380740E942A
:10332000710D83E296E06FE97AE00E94C12A8091F4
:103330009F0380720E94710D83E296E062E87AE05A
:103340000E94C12A8EEB93E00E94EA08AB01BC0107
:1033500083E296E02AE030E00E94A82B83E296E028
:103360006DE77AE00E94C12A8EEB93E00E94EA08A2
:103370009B01AC0160E472E48FE090E00E94F42EC7
:1033800083E296E0BA01A9012AE030E00E94A82B6E
:1033900083E296E06AE77AE00E94002BDF91CF910A
:1033A0001F910895EF92FF920F931F937C0103E208
:1033B00016E0C8016F2D70E04AE050E00E94CB2B70
:1033C000C8016EE20E94E22AB701E4E076956795B3
:1033D000EA95E1F76F707070C8014AE050E00E9412
:1033E000CB2BC8016EE20E94E22A8FE0E822FF2484
:1033F000C801B7014AE050E00E94CB2B1F910F910A
:10340000FF90EF9008950F931F93CF93DF93209138
:10341000EF032F3FA9F583E296E061EF75E00E948C
:10342000C12A83E693E00E94D21983E296E060ED20
:1034300075E00E94C12A8091790490917A040E94DB
:10344000D21983E296E06DE975E00E94002B83E2D9
:1034500096E06AE775E00E94002B83E296E062E660
:1034600075E00E94002B83E296E06DE375E00E9418
:10347000002B83E296E00E94EA2A0E94611769C04D
:1034800012160CF066C0332727FD30958091780422
:1034900090E0821793070CF45CC083E296E068E248
:1034A00075E00E94C12A6091EF03772767FD709550
:1034B00083E296E04AE050E00E945F2C83E296E0CF
:1034C0006DEF74E00E94C12A08E210E03AC0C12FFB
:1034D000D0E0CC0FDD1FC95ADB4F288130E080914E
:1034E000EF03992787FD909501972817390741F534
:1034F00083E296E06FE371E00E94732C83E296E032
:10350000602F4AE050E00E94F02B83E296E063E4F3
:1035100071E00E94732CE981F0E0EF70F070EE0F23
:10352000FF1FE85BFC4F6081718183E296E00E949F
:10353000732C83E296E067E471E00E94732C0F5FC6
:103540001F5F80917704181710F283E296E00E94C3
:10355000EA2ADF91CF911F910F910895ACE1B0E07D
:10356000E4EBFAE10C943B2F282F8091EF038F3F7F
:1035700009F042C1822F90E0FC013A97EF36F10545
:1035800008F033C1EC5CFF4F0C94682F83E296E0A7
:1035900069E471E0AEC083E296E069E471E00E9404
:1035A000762C1CC183E296E065E571E00E94762CE2
:1035B00085E78983DE011296E3EAF3E08BE101906F
:1035C0000D928150E1F7CE0101966CE10E94B50F9A
:1035D0000E94710C83E08093980368EC70E080E0B7
:1035E00090E00E946F2980919803843009F0FDC01B
:1035F0008FE70E94880A0E949C0A8983853509F01A
:10360000F4C083E296E06FED74E00E94002B83E249
:1036100096E061EC74E00E94002B83E296E063EA9E
:1036200074E0ACC083E296E06DE671E00E94762C17
:1036300089E68983CE01019661E00E94B50F0E9460
:10364000710C83E08093980368EC70E080E090E078
:103650000E946F2980919803843009F0C6C08FE7DB
:103660000E94880A0E949C0A89838E010E5F1F4F68
:103670009DE1E92EF12CEC0EFD1E0E949C0AD80162
:103680008D938D01AE15BF05C1F7A3EAB3E0FE012E
:1036900032968BE101900D928150E1F78981893456
:1036A00009F0A3C083E296E065E874E00E94002B75
:1036B00083E296E067E674E00E94002B83E296E0E6
:1036C00069E474E05BC083E296E067E871E00E9421
:1036D000762C8EEF8093EF0388C020522750922FD4
:1036E000905380917804891738F483E296E066E974
:1036F00071E00E94762C79C09093EF036FC084E153
:103700008093EF0383E296E062E174E037C085E1E5
:103710008093EF0383E296E06BED73E02FC086E1C8
:103720008093EF0383E296E064EA73E027C087E1C9
:103730008093EF0383E296E06AE573E01FC088E1BF
:103740008093EF0383E296E069E473E017C089E1B8
:103750008093EF0383E296E065E373E00FC08AE1B4
:103760008093EF0383E296E060E273E007C08BE1B1
:103770008093EF0383E296E068EF72E00E94002BF3
:1037800034C083E296E06EED72E00E94002B8091DF
:10379000B10391E01DC083E296E068EC72E00E9404
:1037A000002B8091B10392E013C083E296E063EBBB
:1037B00072E00E94002B8091B10394E009C083E283
:1037C00096E068E972E00E94002B8091B10398E0D6
:1037D00089278093B1038FEF8093EF030E94031A30
:1037E00004C083E296E00E94F52D83E296E00E94F9
:1037F000BB2D892BB1F763C1822F0E9462168823EB
:1038000009F45DC180915504882321F48FEF8093E2
:10381000EF034DC180EF93E060E070E040E050E0E6
:103820000E94A2069B01AC016091EF03862F9927AD
:1038300087FD9095A92FB92FFC013197EB31F10548
:1038400008F025C1ED55FF4F0C94682FE62FFF2798
:10385000E7FDF0958091780490E08E179F070CF4B7
:1038600016C1DA01C9010197A109B1098097A10523
:10387000B10540F0FF2410E008E26F010894C10890
:10388000D10826C0ED55FC4F822F81508083E7C0C0
:10389000612F70E0660F771F695A7B4FFB018081B3
:1038A00090E08C159D0599F4802F90E0A0E0B0E0A9
:1038B00082179307A407B50749F4F601ED55FC4FAD
:1038C000DB0111968C918183FF24F3940F5F1F5FBE
:1038D000809177041817E0F2C0C02F3F31054105F1
:1038E000510511F008F0D3C02093BB03B8C02F3F9F
:1038F00031054105510511F008F0C9C02093BC0302
:10390000AEC02F3F31054105510511F008F0BFC091
:103910002093BD03A4C08091F0038062803719F525
:1039200081EF93E060E070E040E050E00E94A2068A
:103930009B01AC01DC01CB010197A109B1090897FA
:10394000A105B10508F0B6C0CA01B90124ED30E304
:1039500040E050E00E94C22E9B01AC012A5E3C4A2E
:103960004A46554E24C0863611F581EF93E060E05B
:1039700070E040E050E00E94A2069B01AC01DC0137
:10398000CB010197A109B1090797A105B10508F07D
:1039900091C0CA01B90128EA31E640E050E00E9436
:1039A000C22E9B01AC01245E3C434E46544E211571
:1039B00031054105510561F0DA01C9018054914E8C
:1039C000AD49B8418158904FAA4FB24008F05FC04E
:1039D0002093B3033093B4034093B5035093B603DD
:1039E0003EC02F3F31054105510511F008F04FC091
:1039F0002093B70334C0DA01C9010197A109B109C5
:103A00008F3F9105A105B10508F041C02093B8038F
:103A100026C0DA01C901845C9940A040B0408D54B1
:103A20009D41A040B04038F43093BA032093B903CD
:103A3000FF24F39401C0FF242115310541055105F0
:103A400011F48FEF07C0213131054105510528F4EC
:103A5000822F81508093B20302C0FF20C1F0809179
:103A600056048823D1F48091C7039091C803A09194
:103A7000C903B091CA030196A11DB11D8093C7036C
:103A80009093C803A093C903B093CA0306C083E20E
:103A900096E068EA71E00E94762C0E9458168FEF3B
:103AA0008093EF0383E296E06AE00E94142B0E9469
:103AB000031A05C021E030E040E050E07DCF6C9675
:103AC000E8E00C94572F83E296E06CE472E00E94E9
:103AD000002B83E296E064E372E00E94002B83E215
:103AE00096E00E94BB2D892B31F083E296E00E9484
:103AF000F52D0E94AE1A0E947114823019F08330A5
:103B000069F405C083E296E066E172E004C083E2F6
:103B100096E06FEF71E00E94002B08958FEF809385
:103B2000EF03109256040E94031A0CC083E296E041
:103B30000E94BB2D892B31F083E296E00E94F52D87
:103B40000E94AE1A8091EF038E3F81F70895809115
:103B5000EF03992787FD9095A92FB92FFC01319686
:103B6000EB30F10508F074C0E254FF4F0C94682F5D
:103B700083E296E064E678E00E94002B83E693E01F
:103B80000E94D21983E296E06CE478E00E94002B58
:103B900083E296E067E278E00E94002B83E296E001
:103BA0006DEF77E00E94002B83E296E06CED77E00A
:103BB0000E94002B83E296E06FEA77E00E94002BE0
:103BC00083E296E069E877E00E94002B83E296E0CA
:103BD00065E677E00E94002B83E296E06EE377E0F3
:103BE0000E94002B83E296E00E94EA2A0E94AB1812
:103BF0002FC083E296E061E277E028C083E296E09E
:103C00006CEF76E023C083E296E067EE76E01EC0BC
:103C100083E296E068EC76E019C083E296E064E81F
:103C200076E014C083E296E06FE676E00FC083E2B0
:103C300096E06AE576E00E94002B83E296E064E17C
:103C400076E004C083E296E06EEF75E00E94002B00
:103C50006AE070E080E090E00E946F2904C083E297
:103C600096E00E94F52D83E296E00E94BB2D892B01
:103C7000B1F70895A2E2B0E0E0E4FEE10C94312F48
:103C80008E010F5F1F4F80E1D8011D928A95E9F7E1
:103C900083E296E066EC71E00E94762C0E941D158E
:103CA00020E431EE4DE958E12F8F38A349A35AA300
:103CB00080EC91EDA8E9BBE18B8F9C8FAD8FBE8F1F
:103CC00024EF31E040E050E02F8B388F498F5A8F3E
:103CD00050E5C52E53ECD52EE12CF12C40E4442EBA
:103CE00041EE542E4DE9642E48E1742E8824992427
:103CF000540133241E8A1D8A198A1A8A1B8A1C8A37
:103D0000FFC083E296E00E94F52D8434B9F085343B
:103D100030F48332B9F18C3209F0CCC044C0833521
:103D200009F0C8C02F8D38A149A15AA1C901DA01F3
:103D30002C013D01882499245401E2C083E296E0DD
:103D400064E40E94E22A83E296E040E451EE6DE9E9
:103D500078E12AE030E00E94162C83E296E06CE2E3
:103D60000E94E22A83E296E040EC51ED68E97BE1B3
:103D70002AE030E00E94162C83E296E06CE20E947A
:103D8000142BBEC019821A821B821C821D821E82C5
:103D90001F82188619861A861B861C861D861E861B
:103DA0001F86188A3AC0339434E0331609F0A8C04D
:103DB00069817A818B819C8128EE33E040E050E07C
:103DC0000E94C22E6F8F78A389A39AA36D817E81F2
:103DD0008F8198850E94C22E6B8F7C8F8D8F9E8FD6
:103DE00089859A85AB85BC858F8B988FA98FBA8F73
:103DF0006D857E858F8598890E94C22E6B017C011E
:103E000090E2C9169EE4D90690E0E90690E0F90632
:103E100030F48CE162E30E94B20A332471C0A0E363
:103E2000CA16A5E7DA06A0E0EA06A0E0FA0618F44A
:103E30008CE162E2F0CFB0E4CB16BCE9DB06B0E087
:103E4000EB06B0E0FB0618F48CE166E2E4CFE0E5B7
:103E5000CE16E3ECDE06E0E0EE06E0E0FE0618F447
:103E60008CE162E1D8CFF0E6CF16FAEEDF06F0E0A3
:103E7000EF06F0E0FF0618F48CE165E1CCCF20E717
:103E8000C21621E1D20621E0E20620E0F20618F493
:103E90008CE161E0C0CF30EAC31636E8D30631E0EA
:103EA000E30630E0F30618F48CE163E0B4CF8CE174
:103EB00065E0B1CF30ED232E280E49E0421500F128
:103EC000032D10E0000F111F000F111F81E090E083
:103ED0008C0F9D1F080F191FD8016D917D918D9139
:103EE0009C912AE030E040E050E00E94C22E620D3A
:103EF000711D811D911DF8016083718382839383FD
:103F000083E296E00E94BB2D892B09F0FACE811442
:103F10009104A104B10489F4C301B2010E94280BE9
:103F200061E070E080E090E00E946F29FFEFFE8B7F
:103F30001D8A198A1A8A1B8A1C8A2F89388D498DF5
:103F40005A8D82169306A406B506E0F40E94D30AA1
:103F500029893A894B895C89280F311D411D511DE2
:103F6000298B3A8B4B8B5C8B3D89381708F48D8BF2
:103F70004E89841708F48E8B0894811C911CA11C17
:103F8000B11C56C0C301B20128EE33E040E050E05E
:103F90000E94F42E83E296E0BA01A9012AE030E003
:103FA0000E94A82B83E296E06CE20E94E22A83E260
:103FB00096E06D894AE050E00E94F02B83E296E0A3
:103FC0006CE20E94E22A69897A898B899C89A50121
:103FD00094010E94F42E83E296E0BA01A9012AE03E
:103FE00030E00E94A82B83E296E06CE20E94E22A75
:103FF00083E296E06E894AE050E00E94F02B83E273
:1040000096E06CE20E94142B4C0C5D1C6E1C7F1C15
:104010008B8D9C8DAD8DBE8D84159505A605B70540
:1040200020F44F8C58A069A07AA0882499245401C8
:104030002F8D38A149A15AA1285E334040405040FD
:1040400009F05ECFA296E2E10C944D2FAAE5B0E014
:10405000ECE2F0E20C943D2F8B017A018B3009F4F5
:1040600025C18C3040F5853009F484C0863080F459
:10407000823009F459C0833020F4813009F058C2ED
:1040800042C0833009F461C0843009F051C265C078
:10409000883009F49DC0893038F4863009F486C030
:1040A000873009F045C28CC0893009F499C08A3044
:1040B00009F03EC2C9C0893609F48AC18A3680F443
:1040C000863609F435C1873620F4853609F030C2CA
:1040D00016C1873609F445C1883609F029C249C19D
:1040E0008C3609F4CCC18D3638F48A3609F47BC19C
:1040F0008B3609F01DC2B7C18D3609F4F4C1873C77
:1041000009F016C208C281E069E270E00E946D11F8
:104110000EEB13E0F80181918F010E945611F3E03C
:10412000073E1F07B9F70CC282E06BE170E00E9406
:104130006D1103EA13E0F80181918F010E9456117D
:10414000F3E00E3B1F07B9F7FBC183E061E070E0CD
:104150000E946D110E947114F1C184E061E070E071
:104160000E946D1181E00E9456110E944F110E9421
:104170003A1EE8C16091770470E0660F771F85E012
:104180000E946D1100E010E008C0F801E95AFB4FF1
:1041900080810E9456110F5F1F4F8091770490E03D
:1041A000880F991F0817190780F3CAC186E062E0DB
:1041B00070E00E946D1183E693E00E946411C0C11B
:1041C00087E061E070E00E946D1180917804B6C1D3
:1041D00088E061E070E00E946D1180919903AEC1AA
:1041E00086E68983CE01019661E00E94B50F0E94A8
:1041F000710C83E08093980368EC70E080E090E0BD
:104200000E946F29809198038430E1F48FE70E9427
:10421000880A0E949C0A8983863471F489E060E2EE
:1042200070E00E946D1110E00E949C0A0E945611DD
:104230001F5F1032C9F784C189E061E070E00E941D
:104240006D11CFC089E075C18AE069E070E00E941D
:104250006D1110929A0380918D05882351F0809101
:104260009F039091A003A091A103B091A203806845
:1042700009C080919F039091A003A091A103B091E8
:10428000A2038F7780939F039093A003A093A10331
:10429000B093A2030AE913E0F80181918F010E9413
:1042A0005611F3E0033A1F07B9F74AC18BE061E208
:1042B00070E00E946D118091AC048F3F39F08091C5
:1042C000AC048F5F8093AC04815002C08091AC0439
:1042D0000E94561100E010E0F894F801EE0FFF1F65
:1042E000E95DFC4F808191810E940E0A0E94641159
:1042F00078940F5F1F4F0031110571F721C185E6DA
:1043000061E070E00E946D110932110509F015C1DC
:1043100020E030E0F901E254FC4FD701A20FB31FB7
:104320008C9180832F5F3F4F2932310599F759C017
:1043300086E661E070E00E946D110B31110509F015
:10434000FCC020E030E0F901ED55FC4FD701A20F91
:10435000B31F8C9180832F5F3F4F2B31310599F72D
:1043600040C087E661E070E00E946D110E941A165D
:1043700038C088E661E070E00E946D1185E78A83AD
:10438000DE011396E3EAF3E08BE101900D92815098
:10439000E1F7CE0102966CE10E94B50F0E94710C0C
:1043A00083E08093980360E273E080E090E00E94F5
:1043B0006F2980919803843009F0BFC08FE70E9475
:1043C000880A0E949C0A8A83853509F0B6C009C014
:1043D00089E661E070E00E946D110E944D080E9424
:1043E000920881E0ABC08AE661E070E00E946D1146
:1043F00089E68E8FCE014E9661E00E94B50F0E9435
:10440000710C83E08093980360E273E080E090E0B9
:104410000E946F2980919803843009F08EC08FE745
:104420000E94880A0E949C0A8E8F8E01015E1F4F97
:104430006AE3E62EF12CEC0EFD1E0E949C0AF801A8
:1044400081938F01EE15FF05C1F7A3EAB3E0FE01EA
:104450007F968BE101900D928150E1F78E8D89342A
:1044600009F06BC0BECF8BE661E070E00E946D1179
:10447000F70180810E9448160E942316B2CF8CE675
:1044800061E070E00E946D110032110571F487E661
:104490008AAFDE01DB96F70180E201900D92815038
:1044A000E1F7CE01CA9661E205C087E48AAFCE018A
:1044B000CA9661E00E94B50F0E94710C83E0809360
:1044C00098036CE474E080E090E00E946F29809192
:1044D0009803843091F58FE70E94880A0E949C0A15
:1044E000873459F57ECF8DE661E070E00E946D1152
:1044F0000930110511F520E030E0F901E656FC4FD6
:10450000D701A20FB31F8C9180832F5F3F4F2930BB
:10451000310599F766CF87EC61E070E00E946D117C
:1045200081E00E9456110E944F111092ED030AC0C3
:104530008AEC61E070E00E946D1180E00E945611EB
:104540000E944F11C65ADF4FE6E00C94592FA0E0AD
:10455000B0E0EDEAF2E20C94392F34E0A32E26E02D
:10456000B22E95E0C92E01E215E084E6D82EB2E025
:10457000EB2EA3E0FA2EA1C083E296E00E94F52D77
:10458000982F80938C0580918B05833021F18430A6
:1045900028F4813099F08230B8F409C0853009F4EC
:1045A00048C0853020F1863009F087C05FC0953B58
:1045B00009F083C081E080938B057FC0923609F0BB
:1045C0007AC0E0928B0579C090938A059093890513
:1045D000F0928B0572C090938705109288058091A8
:1045E0008905892780938905A0928B0566C0D92FFC
:1045F000C0E020918705309188052C2B3D2B30930E
:1046000088052093870580918905892780938905EE
:10461000C0928B052536310508F44FC08CEC61E063
:1046200070E00E946D1181E00E9456110E944F11AE
:1046300042C02091850530918605F901EF5DFA4F62
:104640009083809189058927809389052F5F3F4F4B
:104650003093860520938505809187059091880584
:104660002817390750F1B0928B0527C08091890532
:10467000891759F4609185057091860580918A05A6
:1046800041E255E00E9426200DC08BEC62E070E014
:104690000E946D1180918A050E9456118091EE034F
:1046A0000E945611F8018D2D11928A95E9F710920A
:1046B00086051092850510928B0583E296E00E9494
:1046C000BB2D892B09F058CFCDB7DEB7EAE00C94AB
:1046D000552F81E08093ED0308C083E296E00E94AD
:1046E000BB2D892B11F00E94A7228091ED03882316
:1046F000A1F70895A0E0B0E0E0E8F3E20C943C2FCD
:104700000E9449296115710581059105C9F30E942F
:1047100099061092C7031092C8031092C903109211
:10472000CA03DD24E090C703F090C8030091C903D9
:104730001091CA03102F0F2DFE2CEE240E94940618
:104740002FEF30E040E050E00E94162FE60EF71EFB
:10475000081F191FE092C703F092C8030093C90312
:104760001093CA03D39444E0D416E1F6CDECD3E021
:1047700000E010E040E1E42E47E2F42E4EC00F5F6F
:1047800019F40E944D084DC00E94940622E330E0C7
:1047900040E050E00E94162F6F5FEDECF3E090E0F8
:1047A00004C08191861759F39F5F9117D0F38091D0
:1047B000CC0390E08E9D90018F9D300D9E9D300D1D
:1047C0001124862F90E0AC01249FC001259F900DFD
:1047D000349F900D1124AA2797FDA095BA2F209100
:1047E000C3033091C4034091C5035091C603820FA7
:1047F000931FA41FB51F20919B0330919C034091F0
:104800009D0350919E03281739074A075B0708F458
:10481000B6CF69931F5F183121F08881882309F092
:10482000AECFCDB7DEB7E7E00C94582F1F931091B1
:10483000EF031F3F09F0F1C0893409F467C08A34DF
:1048400028F5883309F479C0893368F4803309F492
:1048500086C0813308F06FC08B3109F44DC08132BE
:1048600009F0D5C03DC0813409F49AC0823438F4CF
:10487000893309F472C0803409F0C9C031C0823470
:1048800009F4A1C0863409F0C2C052C0823609F4CE
:104890009AC0833690F4883579F1893538F48235B9
:1048A00009F43FC0833509F0B2C01FC08A3509F44E
:1048B000A9C0813609F0ABC073C0823791F183374C
:1048C00030F48636A9F1893609F0A1C01FC08837B7
:1048D00099F08A3709F496C0833709F098C005C06B
:1048E00083E296E069E471E019C00E941A1683E23F
:1048F00096E063ED71E006C00E94231683E296E025
:104900006DEE71E00E94762C8EEF7FC00E944D0804
:104910000E94920883E296E06CE072E00E94762C9E
:1049200076C00E947A2383E296E065E272E0F6CFD9
:104930000E94CB166CC0805368C083E296E06CEE98
:1049400071E00E94002B9091E603892F885F8871A7
:10495000977E892B8093E60320C089E056C083E2CE
:1049600096E069ED71E00E94002B80919F03909189
:10497000A003A091A103B091A20320E130E040E0A8
:1049800050E082279327A427B52780939F03909315
:10499000A003A093A103B093A2031093EF0337C029
:1049A00083E296E063EC71E00E94002B80919F030C
:1049B0009091A003A091A103B091A20320E430E064
:1049C00040E050E012C083E296E062EB71E00E94AA
:1049D000002B80919F039091A003A091A103B0911F
:1049E000A20320E230E040E050E082279327A42792
:1049F000B52780939F039093A003A093A103B09346
:104A0000A20302C00E94631D8FEF8093EF03809189
:104A1000EF038E3F09F4DDC0D4C00E9462168823E4
:104A200009F4D7C080915504882321F48FEF809337
:104A3000EF03C7C080EF93E060E070E040E050E03B
:104A40000E94A2069B01AC018091EF03992787FD8C
:104A50009095A92FB92FFC013197E930F10508F0A5
:104A60008CC0E753FF4F0C94682FDA01C9018154C1
:104A7000914EAD49B8418F57904FAA4FB24008F0C0
:104A80007CC02093C3033093C4034093C503509369
:104A9000C6039AC02093C7033093C8034093C90349
:104AA0005093CA0381E0809356048EC028303105AC
:104AB0004105510508F061C02093CB0385C0DA01A0
:104AC000C9010197A109B1090A97A105B10508F02B
:104AD00054C02093CC0378C080EF93E06DE371E085
:104AE0000E94BE0710E00EC0183130F4E12FF0E054
:104AF000E254FC4F87871F5F80E090E06DE371E038
:104B00000E94BE07009759F00E94A007009761F726
:104B100006C0E12FF0E0E254FC4F17861F5F18310A
:104B2000C0F352C0253031054105510530F52093C1
:104B3000E5034AC0DA01C9010197A109B109069745
:104B4000A105B105D0F48091E603887F822B809384
:104B5000E6033AC0DA01C9010197A109B109805001
:104B6000924CA140B04048F42093BF033093C0035F
:104B70004093C1035093C20327C083E296E068EAE2
:104B800071E00E94762C13C08091C7039091C803F6
:104B9000A091C903B091CA030196A11DB11D8093D4
:104BA000C7039093C803A093C903B093CA030E949C
:104BB00058168FEF8093EF0383E296E06AE00E943D
:104BC000142B0E94A71D05C0809156048823E1F292
:104BD000EECF1F9108958FEF8093EF03109256044C
:104BE0000E94A71D0CC083E296E00E94BB2D892B7A
:104BF00031F083E296E00E94F52D0E941624809108
:104C0000EF038E3F81F76AE070E080E090E00E9461
:104C10006F2904C083E296E00E94F52D83E296E0BE
:104C20000E94BB2D892BB1F70895AAE2B0E0EBE119
:104C3000F6E20C94362F0E943B297B018C0181E027
:104C40000E94920B04C083E296E00E94F52D83E25D
:104C500096E00E94BB2D892BB1F72D98DD24D394CB
:104C6000E2E67E2E72E0872E912C8C0E9D1E5E0158
:104C70000894A11CB11C63E0C62E0E943B2920E0D1
:104C800030E06E197F09800B910B693C710581053D
:104C9000910510F021E030E08D2D90E0282339239C
:104CA000232B99F10E943B297B018C012C9A80EDEA
:104CB00097E00E94A1117982D401EEEBF3E089E242
:104CC00001900D928150E1F7C5016AE20E94B50F93
:104CD0002C9880E090E00E94A111C09298030E945D
:104CE000710C62E370E080E090E00E946F29809197
:104CF0009803843051F4C09298038FE70E94880A89
:104D00000E949C0A823409F4DD248BE00E946D2A03
:104D1000892B49F5DD24D39426C02D9A2C9A83E261
:104D200096E00E94F52D8D30910569F08E30910549
:104D30001CF40A97B1F407C08332910569F08234FC
:104D4000910579F40CC083E296E064EA71E00E9478
:104D5000002B0E94EB2505C00E943A1E02C00E9453
:104D600069232D982C9883E296E00E94BB2D892B15
:104D700009F483CFD2CF8F929F92AF92BF92CF92FE
:104D8000DF92EF92FF920F931F938BE00E946D2AA8
:104D9000892B09F083C068EC70E080E090E00E940D
:104DA0006F2980E090E00E94A1110E943B295B01E5
:104DB0006C01F0ECEF2EF2E1FF2E012D112DE60E2D
:104DC000F71E081F191F06C08BE00E946D2A892B51
:104DD00009F062C00E943B296E157F05800791078C
:104DE00098F38BE00E946D2A892B09F055C080ED65
:104DF00097E00E94A1110E943B297B018C0199241C
:104E00009394882488E496E2A0E0B0E0A80EB91E4E
:104E1000CA1EDB1E29C0AE14BF04C006D10638F47A
:104E200080ED97E00E94A111882483941DC00E9408
:104E30003B296E197F09800B910B693C7105810537
:104E4000910590F00E943B297B018C0180E0992024
:104E500009F481E0982E882319F480E090E002C0E4
:104E600080ED97E00E94A1118BE00E946D2A892BB2
:104E700091F280E090E00E94A111882049F0809199
:104E800099038F5F83700E9448160E94231606C004
:104E90000E947A230E941A160E9415261F910F91D4
:104EA000FF90EF90DF90CF90BF90AF909F908F904A
:104EB000089580E06DEF77E042E050E00E947628B0
:104EC0000895EF92FF920F931F9380E00E941908BC
:104ED0000E948C118DE061E00E94CE298CE061E09F
:104EE0000E94CE298BE060E00E94CE2983E060E042
:104EF0000E94CE2983E061E00E943A2A8EE061E0C0
:104F00000E94CE298EE060E00E943A2A0E94491455
:104F100083E296E040E052EC61E070E00E94342DC4
:104F20000E943B160E9423160E944F0D8FEF809324
:104F3000AC040E94592778940E943B297B018C0184
:104F40008091AC048F3F09F0C7C00E943B296E19C5
:104F50007F09800B910B605D77408040904008F0A6
:104F6000BBC0EECF83E296E00E94F52D83E296E08F
:104F70000E94BB2D892BB1F783E296E062E472E0D8
:104F80000E94732C83E693E00E94D21983E296E09C
:104F900069E572E00E94732C83E296E062E070E0C3
:104FA0004AE050E00E945F2C62E370E080E090E015
:104FB0000E946F2983E296E00E94BB2D04970CF1BA
:104FC00083E296E00E94F52D82349105D1F483E2CC
:104FD00096E00E94F52D8E34910599F483E296E0D7
:104FE0000E94F52D8434910561F483E296E00E94DD
:104FF000F52D819731F480E090E00E94A1110E948C
:1050000015264091BF035091C0036091C103709178
:10501000C203DB01CA010197A109B1090497A105E7
:10502000B10568F44093AD04433029F040E052EC00
:1050300061E070E004C040EA56E861E070E083E2BD
:1050400096E00E94342D0E94BB262D9880E090E0CF
:105050000E94A1110E944F0D80E00E94920B80914E
:1050600092040E94BD0A0E94710C109215051092C4
:1050700016051092170510E015C062E370E080E09D
:1050800090E00E946F2980ED97E00E94A11162E3F9
:1050900070E080E090E00E946F2980E090E00E9444
:1050A000A1111F5F80919903811738F78091E60362
:1050B00090E084FF09C020E088719070489709F45F
:1050C00021E0822F0E9452148FE00E9419081F9144
:1050D0000F91FF90EF90089580ED97E00E94A1114D
:1050E0008BE061E00E943A2A2D9A40CF823000F591
:1050F000E82FF0E0EE0FFF1FE257FA4F7183608355
:10510000882319F08130A1F408C0809169008C7F58
:10511000842B80936900E89A089580916900440F78
:10512000551F440F551F837F842B80936900E99A94
:1051300008951F920F920FB60F9211242F933F9351
:105140004F935F936F937F938F939F93AF93BF938F
:10515000EF93FF9380918E0590918F05892B29F015
:10516000E0918E05F0918F050995FF91EF91BF9128
:10517000AF919F918F917F916F915F914F913F91EF
:105180002F910F900FBE0F901F9018951F920F92A6
:105190000FB60F9211242F933F934F935F936F930A
:1051A0007F938F939F93AF93BF93EF93FF938091E0
:1051B000900590919105892B29F0E0919005F0914F
:1051C00091050995FF91EF91BF91AF919F918F91BB
:1051D0007F916F915F914F913F912F910F900FBEF3
:1051E0000F901F9018951F920F920FB60F921124D7
:1051F0002F933F938F939F93AF93BF938091960587
:1052000090919705A0919805B091990530919A05D4
:105210000196A11DB11D232F2D5F2D3720F02D5795
:105220000196A11DB11D20939A0580939605909338
:105230009705A0939805B093990580919205909158
:105240009305A0919405B09195050196A11DB11DFE
:105250008093920590939305A0939405B093950540
:10526000BF91AF919F918F913F912F910F900FBE62
:105270000F901F9018958FB7F89420919605309154
:10528000970540919805509199058FBFB901CA01C2
:1052900008959FB7F894209192053091930540911D
:1052A00094055091950586B5A89B06C08F3F21F0C7
:1052B0002F5F3F4F4F4F5F4F9FBF542F432F322FD2
:1052C0002227280F311D411D511D82E0220F331F5F
:1052D000441F551F8A95D1F7B901CA010895EF926D
:1052E000FF920F931F93CF93DF937B018C010E945A
:1052F0004929EB010EC00E9449296C1B7D0B685E99
:105300007340C8F30894E108F10801091109C85174
:10531000DC4FE114F1040105110569F7CDB7DEB7E3
:10532000E6E00C94592F789484B5826084BD84B5EE
:10533000816084BD85B5826085BD85B5816085BD90
:10534000EEE6F0E0808181608083E1E8F0E01082A9
:10535000808182608083808181608083E0E8F0E0EA
:10536000808181608083E1EBF0E0808184608083D4
:10537000E0EBF0E0808181608083EAE7F0E080810B
:10538000846080838081826080838081816080836B
:105390008081806880831092C1000895CF93DF934D
:1053A000482F50E0CA018D5F934FFC013491415169
:1053B000544FFA018491882369F190E0880F991F76
:1053C000FC01EF52F44FA591B491FC01E552F44F6A
:1053D000C591D491662351F42FB7F8948C91932FF3
:1053E000909589238C93888189230BC0623061F466
:1053F0002FB7F8948C91932F909589238C93888163
:10540000832B88832FBF06C09FB7F8948C91832B82
:105410008C939FBFDF91CF910895833071F08430DA
:1054200028F48130A1F0823021F514C08630B1F02B
:105430008730D1F08430E9F404C0809180008F7708
:1054400003C0809180008F7D80938000089584B593
:105450008F7702C084B58F7D84BD08958091B000A0
:105460008F778093B00008958091B0008F7D8093F6
:10547000B0000895FF920F931F93F62E482F50E02F
:10548000CA01895E934FFC012491CA018D5F934F3D
:10549000FC0114914151544FFA0104910023C9F0C9
:1054A000222319F0822F0E940D2AE02FF0E0EE0F48
:1054B000FF1FE552F44FA591B4919FB7F894FF20D8
:1054C00021F48C911095812302C08C91812B8C93B7
:1054D0009FBF1F910F91FF9008950F931F93482F27
:1054E00050E0CA01895E934FFC012491CA018D5F8F
:1054F000934FFC0104914151544FFA01149111232F
:1055000019F420E030E015C0222319F0822F0E9408
:105510000D2A812F90E0880F991F8B51944FFC0129
:10552000A591B4918C9120E030E0802311F021E02E
:1055300030E0C9011F910F910895A0E0B0E0E3EAC7
:10554000FAE20C943B2F7C016B018A01C0E0D0E0B1
:105550000FC0D6016D916D01D701ED91FC910190C5
:10556000F081E02DC7010995C80FD91F01501040E7
:105570000115110571F7CE01CDB7DEB7E8E00C9447
:10558000572FEF92FF920F931F93CF93DF937C01DE
:105590008B01C0E0D0E0F8010F5F1F4F64916623DC
:1055A00059F0D701ED91FC910190F081E02DC701F8
:1055B0000995C80FD91FEFCFCE01CDB7DEB7E6E012
:1055C0000C94592FDC01ED91FC910190F081E02DBC
:1055D00009950895EF92FF920F931F938C016DE050
:1055E0000E94E22A7C01C8016AE00E94E22A9C0132
:1055F0002E0D3F1DC9011F910F91FF90EF9008954F
:10560000EF92FF920F931F937C010E94C12A8C019D
:10561000C7010E94EA2A9C01200F311FC9011F9176
:105620000F91FF90EF900895EF92FF920F931F93C9
:105630007C010E94E22A8C01C7010E94EA2A9C0197
:10564000200F311FC9011F910F91FF90EF90089516
:10565000CF93DF93EC016115710519F420E030E080
:105660000FC0DB010D900020E9F71197A61BB70BC7
:10567000E881F9810280F381E02DAD0109959C015B
:10568000C901DF91CF9108954F925F927F928F92DF
:105690009F92AF92BF92CF92DF92EF92FF920F93C1
:1056A0001F93DF93CF93CDB7DEB7A1970FB6F894D2
:1056B000DEBF0FBECDBF2C01742ECB01223008F40B
:1056C0002AE019A231E2C32ED12CCC0EDD1E822E8F
:1056D0009924AA24BB24672D752FA50194010E944B
:1056E000F42E79018A01C801B701A50194010E9435
:1056F000C22E472D461B0894C108D1084A3010F429
:10570000405D01C0495CF6014083E114F1040105EC
:10571000110521F07E2C5F2DC801DDCFC201B6013D
:105720000E94282BA1960FB6F894DEBF0FBECDBF06
:10573000CF91DF911F910F91FF90EF90DF90CF906D
:10574000BF90AF909F908F907F905F904F90089503
:10575000DC012115310541F4ED91FC910190F081BE
:10576000E02D642F099508950E94442B0895EF922F
:10577000FF920F931F937C010E94A82B8C01C701FD
:105780000E94EA2A9C01200F311FC9011F910F912D
:10579000FF90EF900895EF92FF920F931F939A015D
:1057A0007B0100E010E0B801A7010E94A82B1F9127
:1057B0000F91FF90EF900895EF92FF920F931F9338
:1057C0007C010E94CB2B8C01C7010E94EA2A9C011C
:1057D000200F311FC9011F910F91FF90EF90089585
:1057E000EF92FF920F931F939A01E62EFF2400E0A1
:1057F00010E0B801A7010E94A82B1F910F91FF9004
:10580000EF900895EF92FF920F931F937C010E94F7
:10581000F02B8C01C7010E94EA2A9C01200F311F46
:10582000C9011F910F91FF90EF900895A0E0B0E0A3
:10583000ECE1FCE20C943B2FEC016A017B012115A9
:10584000310541F4E881F9810190F081E02D642F68
:1058500009951BC02A303105B1F477FF13C06DE202
:105860000E94E22A8C0144275527BA014C195D0990
:105870006E097F09CE012AE00E94442B9C01200F73
:10588000311F04C02AE00E94442B9C01C901CDB7FE
:10589000DEB7E8E00C94572FEF92FF920F931F931F
:1058A0007B019A010027F7FC0095102FB801A70192
:1058B0000E94162C1F910F91FF90EF900895EF9288
:1058C000FF920F931F937C010E944C2C8C01C70107
:1058D0000E94EA2A9C01200F311FC9011F910F91DC
:1058E000FF90EF9008950E94282B0895EF92FF9269
:1058F0000F931F937C010E94732C8C01C7010E949F
:10590000EA2A9C01200F311FC9011F910F91FF90BE
:10591000EF90089508951F920F920FB60F921124E1
:105920002F933F934F938F939F93EF93FF93809188
:10593000C00082FD1DC04091C6002091DB05309162
:10594000DC052F5F3F4F2F7330708091DD05909104
:10595000DE052817390771F0E091DB05F091DC05D1
:10596000E556FA4F40833093DC052093DB0502C0F7
:105970008091C600FF91EF919F918F914F913F9140
:105980002F910F900FBE0F901F9018951F920F929E
:105990000FB60F9211242F933F938F939F93EF9302
:1059A000FF9320911F06309120068091210690914F
:1059B00022062817390731F48091C1008F7D80932A
:1059C000C10014C0E0912106F0912206E152FA4F85
:1059D0002081809121069091220601968F7390700C
:1059E00090932206809321062093C600FF91EF91A9
:1059F0009F918F913F912F910F900FBE0F901F900D
:105A00001895A0E0B0E0E7E0FDE20C94372FFC0130
:105A10001382128288EE93E0A0E0B0E08483958345
:105A2000A683B7838AE893E0918380837587648730
:105A300057874687318B208B138B028BF58AE48A3C
:105A4000D78AC68AB18EA08E938E828E8F85848FE0
:105A50008889858F8989868F8A89878F8B8980A39A
:105A60002096ECE00C94532FAF92BF92DF92EF920E
:105A7000FF920F931F93CF93DF93EC017A018B0179
:105A8000DD24403081EE580780E0680780E0780729
:105A900011F0DD24D39491E0A92EB12CEC89FD897D
:105AA000DD2069F0C50108A002C0880F991F0A9483
:105AB000E2F7808360E079E08DE390E005C010823A
:105AC00060E874E88EE190E0A80197010E94F42E4E
:105AD0002150304040405040569547953795279586
:105AE00080E12030380720F0DD2011F0DD24D6CF12
:105AF000E889F9893083EA89FB89208319A2EE8934
:105B0000FF89408121E030E0C9010C8C02C0880F80
:105B1000991F0A94E2F7482B4083EE89FF89408160
:105B2000C9010D8C02C0880F991F0A94E2F7482B17
:105B30004083EE89FF894081C9010E8C02C0880F25
:105B4000991F0A94E2F7482B4083EE89FF898081F0
:105B50000F8C02C0220F331F0A94E2F720952823EE
:105B60002083DF91CF911F910F91FF90EF90DF90F5
:105B7000BF90AF900895DC011C96ED91FC911D97AC
:105B8000E05CFF4F2191319180819181281B390B7D
:105B90002F733070C901089583E296E00E94BB2DF7
:105BA000892B11F00E948A2C0895DC011C96ED913E
:105BB000FC911D97E05CFF4F20813181E054F04063
:105BC000DF01AE5BBF4F8D919C911197281739076C
:105BD00019F42FEF3FEF07C08D919C91E80FF91F4B
:105BE0008081282F30E0C9010895DC011C96ED91D9
:105BF000FC911D97E05CFF4F20813181E054F04023
:105C0000DF01AE5BBF4F8D919C911197281739072B
:105C100019F42FEF3FEF10C08D919C911197E80F71
:105C2000F91F20818D919C91119701968F7390702F
:105C300011969C938E9330E0C9010895DC019196F2
:105C40008C919197882339F05496ED91FC9155975A
:105C5000808186FFF9CF91961C920895CF93DF93B0
:105C6000EC01EE85FF85E05CFF4F20813181E0543F
:105C7000F0402F5F3F4F2F733070DF01AE5BBF4F9F
:105C80008D919C91119728173907D1F3E05CFF4F54
:105C900080819181E054F040E80FF91F6083EE8528
:105CA000FF85E05CFF4F31832083EE89FF892081EF
:105CB00081E090E00F8C02C0880F991F0A94E2F7F0
:105CC000282B208381E089A3EC89FD898081806471
:105CD000808381E090E0DF91CF9108958F929F9231
:105CE000AF92BF92CF92DF92EF92FF920F931F93EA
:105CF00000D000D00F92EDB7FEB7319684E0ADB77B
:105D0000BEB711968C9383E0818387E0828385E020
:105D1000838381E0848383E296E06BE975E04FED55
:105D200055E025EC30E004EC10E0B0ECEB2EF12C6B
:105D3000A1ECCA2ED12CF2ECAF2EB12CE6EC8E2EBB
:105D4000912C0E94012D0F900F900F900F900F90AB
:105D50001F910F91FF90EF90DF90CF90BF90AF9089
:105D60009F908F900895CF93DF930E9493290E9474
:105D70006127CCECDDE20E94AB112097E1F30E9499
:105D8000CC2DF9CF629FD001739FF001829FE00D6F
:105D9000F11D649FE00DF11D929FF00D839FF00DAA
:105DA000749FF00D659FF00D9927729FB00DE11D56
:105DB000F91F639FB00DE11DF91FBD01CF01112433
:105DC000089597FB092E07260AD077FD04D086D0C8
:105DD00006D000201AF4709561957F4F0895F6F76C
:105DE000909581959F4F0895A1E21A2EAA1BBB1B87
:105DF000FD010DC0AA1FBB1FEE1FFF1FA217B30797
:105E0000E407F50720F0A21BB30BE40BF50B661FAC
:105E1000771F881F991F1A9469F760957095809570
:105E200090959B01AC01BD01CF01089597FB092E10
:105E300005260ED057FD04D0D7DF0AD0001C38F459
:105E400050954095309521953F4F4F4F5F4F0895A6
:105E5000F6F790958095709561957F4F8F4F9F4F86
:105E600008952F923F924F925F926F927F928F92FE
:105E70009F92AF92BF92CF92DF92EF92FF920F93D9
:105E80001F93CF93DF93CDB7DEB7CA1BDB0B0FB6E3
:105E9000F894DEBF0FBECDBF09942A8839884888A0
:105EA0005F846E847D848C849B84AA84B984C88436
:105EB000DF80EE80FD800C811B81AA81B981CE0F2D
:105EC000D11D0FB6F894DEBF0FBECDBFED01089512
:105ED000EE0FFF1F0590F491E02D0994AA1BBB1B48
:105EE00051E107C0AA1FBB1FA617B70710F0A61BDA
:105EF000B70B881F991F5A95A9F780959095BC01FB
:105F0000CD010895911106C0803219F08950855055
:0E5F1000D0F70895992788270895F894FFCFB9
:105F1E004E6F005965730054582074696D656F7526
:105F2E007421006D6F64756C65206C6F636B6564B6
:105F3E003F00486F70206368616E6E656C200020B4
:105F4E0040200053004E2F4100386368002C002C77
:105F5E00205B005D20280029004E4F5420454E4105
:105F6E00424C45440053656E64696E6720736574D8
:105F7E0074696E677320746F2052580A00526573ED
:105F8E00657474696E672073657474696E677320C7
:105F9E006F6E2052580A0041626F727465642065FC
:105FAE00646974730A00696E76616C696420736546
:105FBE006C656374696F6E000D0A496E76616C696B
:105FCE006420696E707574202D206469736361722C
:105FDE006465642107007363616E6E6572206D6F78
:105FEE0064650053657474696E67732073617665BA
:105FFE006420746F20454550524F4D0A005265760D
:10600E0065727465642073657474696E6773206657
:10601E00726F6D20454550524F4D0A004C6F6164B2
:10602E00656420666163746F72792064656661755C
:10603E006C74730A004B657920616E64206368612D
:10604E006E6E656C732072616E646F6D697A6564D5
:10605E000A004F70656E4C52536E67205458207371
:10606E0074617274696E672000206F6E204857202D
:10607E000050504D00525353490053444100534376
:10608E004C00525844005458440041494E004C4272
:10609E004545500053504B54524D005342555300FA
:1060AE0053554D44004C4C494E440000342B3400A3
:1060BE003800382B340031320031322B3400313677
:1060CE000001000000C01200001A400AA1204EA5D7
:1060DE00001B1E27522C23308025000005400AA1EC
:1060EE00204EA50020244EA52C2330004B00000688
:1060FE00400AD0009D49007B289D492C233000E1A9
:10610E00000005400A4501D7DC03B81E0EBF002370
:10611E002E48E801008A400A6001555502AD1E2046
:10612E00000023C88025000005400AA1204EA500CE
:10613E0020244EA52C233000020002000200020093
:10614E000200020002000200020002000200020031
:10615E0002000200020002FF610265026A026E0284
:10616E00720276027A027E0284028B0290029502FD
:10617E009B029B029B029B0235019C02A002A20283
:10618E00A602A902AE02350100070B0C1011150074
:10619E00160A13223129000000002E2E9D2ABB2D37
:0661AE00F52DD52D1E2E7B
:00000001FF
